:10000000E4C0FEC0FDC0FCC0FBC0FAC0F9C0F8C02F
:10001000F7C0F6C0F5C0F4C0F3C0F2C0F1C0F0C044
:10002000EFC0EEC0EDC014C223C239C2F8C5F7C597
:1000300065C261C3F4C5F3C5F2C5F1C5F0C5EFC52E
:10004000EEC5EDC5A0C20CC30FC3FFC1FBC12EC3DB
:10005000EBC47AC58CC578C58AC589C588C5A7C5CE
:10006000E9C52AC2DCC5DBC5DAC5D9C5D8C5D7C53F
:10007000D6C5D5C5D4C5D3C5D2C5D1C5D0C5CFC5C4
:100080001DC21EC220C2CBC521C222C22BC214C2B5
:1000900021C2C5C529C2C3C5C2C5CCC51DC21FC2A8
:1000A0001B5B306D1B5B324A1B5B303B3066005480
:1000B00068616E6B20796F752E2E2E313031330DC5
:1000C0000A0059454F455549204279207777772EC8
:1000D000426F6172644C61622E6E65740D0A004A53
:1000E00075737420636C6F73652074686520656434
:1000F00069746572204E6F207265736574206E6539
:10010000656465642E0D0A004156525F49535020C4
:1001100053544B3530302052656164792021210DD4
:100120000A0D0A002028686578290D0A000D0A4F7B
:100130004B7E21212053572076657273696F6E20A4
:100140006973206E6F773A20005D3A200050726527
:100150007373204B6579204D696E6F7220696E2034
:10016000686578205B005D3A2000507265737320EB
:100170004B6579204D616A6F7220696E20686578E1
:10018000205B00426F617264204C6162202D2077F9
:1001900077772E426F6172644C61622E6E657420B7
:1001A0002D0D0A0D0A004156525F4953505F5354BA
:1001B0004B3530305F56322056657273696F6E2052
:1001C0004564697465720D0A000011241FBECFE5F5
:1001D000D4E0DEBFCDBF10E0A0E6B0E0E6E7F0E19E
:1001E00002C005900D92AC36B107D9F711E0ACE62C
:1001F000B0E001C01D92A03AB107E1F71DD539C7A3
:10020000FFCE8BE1C3D585E4C1D50895DF92EF928F
:10021000FF920F931F93882319F022E0E22E02C071
:10022000EE24E39481E0CFD5182F92E0D92E0FEF82
:100230002DC080EDF82EF10E89E08F1538F4812F56
:100240008154863018F080528630E8F40F3F09F46C
:1002500000E0812F9BD589E08F1520F00295007F6B
:100260000F0D10C0812F8154863030F4802F82957D
:10027000807F012F075305C0802F8295807F012F3B
:100280000755080FDA9481E09ED5182F1D3039F0FC
:100290001A3029F0DD2069F603C081E094D5EA9494
:1002A000EE20D9F7802F1F910F91FF90EF90DF90F4
:1002B00008951F93182F80EA90E076D586EA91E0A2
:1002C00073D583E891E070D58AE691E06DD5809191
:1002D0009E0190E066E770E040E150E07DD686E761
:1002E00090E058D586E691E05FD5812F8FDF8F3F74
:1002F00011F080939E0185DF8DE491E055D58091CA
:100300009F0190E066E770E040E150E065D686E747
:1003100090E040D589E491E047D5812F77DF8F3F8A
:1003200011F080939F016DDF81E090E060919F016B
:100330006FD682E090E060919E016AD680E090E006
:1003400064E166D68DE291E02FD580919E0190E028
:1003500066E770E040E150E03FD686E790E01AD5CE
:100360008EE214D580919F01803110F480E30ED588
:1003700080919F0190E066E770E040E150E02CD66C
:1003800086E790E007D584E291E00ED588E091E021
:100390000BD58FED90E008D582EC90E005D58FEA83
:1003A00090E002D51F910895A1E0B0E0E9EDF1E001
:1003B000DFC5D82E7B01CB0101978D51914030F0E4
:1003C00080EC8093770042E0E42EF12C8BE1DED4C8
:1003D0008D2DDCD48F2DDAD48E2DD8D48EE0D6D4CA
:1003E00095E19D259E259F259983B6D536E7C32E99
:1003F00030E0D32E87010C0D1D1D998109C0F60137
:1004000080819983C3D4F60181916F0199819827E6
:10041000C016D106A1F7892FB9D42196E8E0C4C54A
:10042000A0E0B0E0E5E1F2E099C5282E80917600E9
:1004300090E0FC013197ED31F10508F0F0C3ED5E7D
:10044000FF4F0994DD24D394F0C2552453942FC157
:1004500081E0809376001092770088E080937800A6
:1004600089E790E060E670E0B0D56BE070E0DCC357
:1004700080917700883921F480917800AED480C0D3
:100480008E3929F4809178008093690079C08F3982
:1004900009F076C08091780080936C0071C08091E3
:1004A000770090E0FC01E058F040E032F10508F000
:1004B000B6C3E05DFF4F099481E01BC08FE019C017
:1004C00080919E0113C080919F0110C082E311C0F2
:1004D00089E10FC0A5D40AC08091690007C080914E
:1004E0006C0004C082E005C08CE803C08F3F09F4B3
:1004F00096C3109277008093780036C3609177009E
:1005000070917800272F30E040E050E0A9013327B8
:100510002227862F90E0A0E0B0E0B82FAA279927E5
:100520008827282B392B4A2B5B2B8091790090E070
:10053000A0E0B0E0BA2FA92F982F8827282B392BBD
:100540004A2B5B2B80917A0090E0A0E0B0E0282B52
:10055000392B4A2B5B2B20936D0030936E00409318
:100560006F005093700067FF04C081E080937100BA
:1005700002C0109271007093720081E0809373004A
:10058000109277004FC3A898A99ABAD480917800A6
:1005900090E0CED480EC8093770080917A00813314
:1005A00018F080E380937A0080917B00882319F40F
:1005B00081E080937B00C0E0D0E04AC0CDD4A89811
:1005C0008091790090E0B4D480917E003AD48091FB
:1005D0007B0090E0ADD480917F0033D480917B008C
:1005E00090E0A6D4A89A809180002BD4182F8091F7
:1005F0007B0090E09DD48091810023D4982F80913E
:100600007D00833031F480917C00181711F4109232
:10061000770080917D00833031F080917C009817C5
:1006200011F41092770080917D00882311F41092CC
:10063000770080917700882331F4A89880917A0020
:10064000C82FD0E005C02196EED384E190E070D4AD
:1006500080917A0090E0C817D90708F4AFCFE2C2C2
:100660003CD4A89AA9988CCF80917900EAD3809144
:100670007A00E7D380917B00E4D380917C00E1D3C2
:1006800080917800882311F016E906C080917700E8
:1006900090E04ED475CF115060E070E080E090EFB4
:1006A00001D480FF6DCF1123B1F76ACF552480911B
:1006B0007A00843018F484E080937A0080917A0084
:1006C000813218F080E280937A0080916D009091E1
:1006D0006E0090937500809374009091770080E095
:1006E00020917800622E7724682A792A29E16216FF
:1006F00021E0720610F080EC93C22ED44090790075
:1007000040FE0AC060E8C62E60E0D62EEE24FF242C
:100710008701C0E0D0E026C150E8A52E50E0B52EFC
:1007200046E9D42ECC24EE24FF248701C0E0D0E09B
:1007300032E0332E8DC0552031F0C0FF04C08091CF
:100740007B00886002C080917B007BD380916D002C
:1007500090916E009FD3D5018C9173D390917E00C0
:10076000F5018081981799F0E0906D00F0906E008F
:1007700000916F00109170008FEF9FEFA0E0B0E04C
:10078000E822F9220A231B234092790002C030920A
:100790007900E2D3552019F482E090E0C9D380912A
:1007A000790082FF22C090917E0026E9D22E81E05E
:1007B000882E912C8C229D2211C0552031F088204A
:1007C00021F080917D00886002C080917D0039D346
:1007D000C70160D380E035D3982FDA9480917E00F2
:1007E0009817B9F4DD2049F714C083FF0EC0B6E9AD
:1007F000DB2E01C0DA9460E070E080E090EF52D32D
:1008000080FF07C0DD20B1F704C080917A0090E03E
:100810008FD3552011F0C0FF13C080916D009091CF
:100820006E00A0916F00B09170000196A11DB11DE6
:1008300080936D0090936E00A0936F00B093700052
:10084000DD2011F4A0E8CA2E21960894A11CB11C49
:10085000C615D70508F46FCFE4C07ED38091710030
:100860008823A9F080916D0090916E00892B21F072
:1008700080917300882359F08DE4E3D280E0E1D2C7
:1008800080917200DED280E0DCD21092730055209D
:1008900031F0C0FF04C080917B00886002C080916D
:1008A0007B00CFD280916D0090916E00F3D2D60183
:1008B0008C91C7D290917E00F6018081981789F0C3
:1008C000E0906D00F0906E0000916F00109170004C
:1008D0008FEF9FEFA0E0B0E0E822F9220A231B236C
:1008E00006C08091790080788061809379005520DE
:1008F00011F1C0FF33C080916D0090916E00A09106
:100900006F00B09170000196A11DB11D80936D0024
:1009100090936E00A0936F00B0937000A070B070C1
:100920008F5F9F4FA040B040C9F4809172008F5FED
:100930008093720013C080916D0090916E00A09121
:100940006F00B09170000196A11DB11D80936D00E4
:1009500090936E00A0936F00B0937000219608945E
:10096000C11CD11CC615D70508F477CFF5D28091EC
:10097000790087FF4FC080917C0063D28091740022
:100980009091750087D280E05CD2552019F481E007
:1009900090E0CED28091790085FF26C0E114F10469
:1009A0000105110509F190917E00F6E9DF2EE701BE
:1009B000C170D0700FC0209721F080917D008860B9
:1009C00002C080917D003DD2C70164D280E039D25F
:1009D000982FDA9480917E00981719F4DD2059F74A
:1009E0001BC0DD20C9F016C086FF10C016E901C08B
:1009F000115060E070E080E090EF54D280FF03C0BF
:100A00001123B1F70CC0112351F004C080917A007A
:100A100090E08ED2CC2405C0E0E8CE2E02C071E872
:100A2000C72EC0927700FEC0DD249091770080E051
:100A300020917800C22FD0E0C0907900C82BD92B2C
:100A4000F1E0C931DF0710F0C8E1D1E068E7E62E38
:100A500060E0F62E00E010E058E0B52EBC2867C03C
:100A60007BD2809171008823A9F080916D009091D4
:100A70006E00892B21F080917300882359F08DE45A
:100A8000E0D180E0DED180917200DBD180E0D9D16D
:100A900010927300DD2021F000FF02C08B2D01C0F9
:100AA0008C2DCFD180916D0090916E00F3D180E0BC
:100AB000C8D1D7018C93DD2011F100FF33C08091A4
:100AC0006D0090916E00A0916F00B0917000019642
:100AD000A11DB11D80936D0090936E00A0936F00D7
:100AE000B0937000A070B0708F5F9F4FA040B04077
:100AF000C9F4809172008F5F8093720013C080915F
:100B00006D0090916E00A0916F00B0917000019601
:100B1000A11DB11D80936D0090936E00A0936F0096
:100B2000B09370000F5F1F4F0894E11CF11C0C176D
:100B30001D0708F495CFBE016D5F7F4F10927700BF
:100B4000CA58DF4F1A8270C0809177007AD18091A5
:100B5000780077D18091790074D180917A0071D139
:100B6000109277001092780063E070E05DC008E7B3
:100B700010E0C1E0D0E0D8018C9163D1282F8091A2
:100B8000770090E08C179D0711F42093780085E0A2
:100B900090E0CED10F5F1F4F2196C530D10559F798
:100BA000109277001092790064E070E03DC0F09000
:100BB0007800E090790010E000E01BC085E090E054
:100BC000B7D10E1578F01F1568F4E02FF0E0EA5861
:100BD000FF4F848136D1E12FF0E0EA58FF4F828346
:100BE0001F5F06C0E02FF0E0EA58FF4F848129D153
:100BF0000F5F80917700081708F304C0EA58FF4F91
:100C000012821F5FE12FF0E01F15C0F3BF016D5F7F
:100C10007F4F10927700EA58FF4F128205C089EC8F
:100C20008093770062E070E0822DBEDBCDB7DEB747
:100C3000E2E1B0C180E05DCCA0E0B0E0E1E2F6E04E
:100C400095C19CD07FD1A09AA19AA89AA99878948E
:100C50008AE080939F0182E080939E0180E090E093
:100C6000CFD1843151F481E090E0CAD180939F01CB
:100C700082E090E0C5D180939E01AA2402C0C12EDB
:100C800006C0BB24EE24FF24C0E0D0E0CC2481E0E9
:100C90009AD0182F8B3149F401E0BBE1DB2E80E0C4
:100CA00092D0182F013009F51CC08D3011F08A3018
:100CB00041F72196AA2039F41A3051F48DE0C81674
:100CC00039F4AA24A394C430D105C9F681E004C044
:100CD000C230D105A1F680E0ECDAC12EC0E0D0E050
:100CE000D6CFD826B82E02E0DACF023029F4D826A3
:100CF000F82EEE2403E0D3CF033031F4D82690E071
:100D0000E82AF92A04E0CBCF043041F4D8268E300B
:100D100009F0BDCF05E0C0E0D0E0C1CF0530B9F4A7
:100D2000CE15DF050CF0ADCF81E0C831D8070CF04F
:100D3000A8CFD126FE01EA58FF4F10832196A8952F
:100D4000CE15DF0509F0ABCF7E0106E0A8CF063057
:100D500009F097CF8D1539F41E141F0424F4A895BB
:100D60008B2D5EDB8ECF80EB8093760081EC8093C1
:100D700077008B2D62E070E017DB83CF10BC81E041
:100D800089B988E18AB986E880BD08955D9BFECF68
:100D90008CB90895FC0104C05D9BFECF8CB93196DF
:100DA00080818823C9F7089503C05D9BFECF2CB9CD
:100DB000FC01019624912223C1F7089501C08CB152
:100DC0005F99FDCF08951F93182F02C01111C4D051
:100DD0005F9BFCCF8CB11F91089510929D018430D0
:100DE00028F081E080939D018CE010C0833019F4DD
:100DF0007098699A0AC0823021F47098699A68984C
:100E000005C0813031F470986998689A80936A00BF
:100E1000089570986898699810926A0080E0089523
:100E200080916A0008952DB11DB8C5988CE590E0B9
:100E3000FC013197F1F7C59A0197F1F7C5982DB9E3
:100E40000895E82F80919D01882329F4EFB9779BBD
:100E5000FECF5FB11DC0C59840E850E020E030E013
:100E60006CE570E0842F8E2311F0C39A01C0C39803
:100E7000CB010197F1F7B499542BC59ACB01019797
:100E8000F1F7C59846952F5F3F4F2830310551F750
:100E9000852F08951F93182F892FD3DF812FD1DF3E
:100EA0001F910895EF92FF920F931F937B018C0186
:100EB000892F9927AA27BB27C4DFC801AA27BB27E8
:100EC000C0DFBB27A12F902F8F2DBBDF8E2DB9DF69
:100ED0001F910F91FF90EF9008951DB8C29ABB9893
:100EE000C398BD98C598BA98C2980895C29A8CE5DF
:100EF00090E00197F1F7C29884E190E019D008954D
:100F0000BA9AC29ABB9AC398BD9AC59884E190E0F8
:100F10000FD080919D01882329F481E58DB98091BE
:100F20006A005BDFC29884E190E002D0DFDF0895C1
:100F300024E733E004C0F9013197F1F701970097F6
:100F4000D1F708952FE088E190E00FB6F894A895C6
:100F500081BD0FBE21BD0895A89508952F923F929F
:100F60004F925F926F927F928F929F92AF92BF92B9
:100F7000CF92DF92EF92FF920F931F93CF93DF9365
:100F8000CDB7DEB7CA1BDB0B0FB6F894DEBF0FBEC2
:100F9000CDBF09942A88398848885F846E847D840F
:100FA0008C849B84AA84B984C884DF80EE80FD8011
:100FB0000C811B81AA81B981CE0FD11D0FB6F89487
:100FC000DEBF0FBECDBFED010895FB01DC01019036
:100FD0000D920020E1F70895FB019F0142306CF073
:100FE00045325CF4642F772730D0805D8A330CF073
:100FF000895D8193CB010097A9F71082C90115C0C3
:10100000E199FECF9FBB8EBBE09A99278DB30895DF
:10101000262FE199FECF9FBB8EBB2DBB0FB6F89458
:10102000E29AE19A0FBE01960895DC01FC01672F58
:1010300071917723E1F7329704C07C916D937083AF
:101040006291AE17BF07C8F30895AA1BBB1B51E1FD
:1010500007C0AA1FBB1FA617B70710F0A61BB70B28
:10106000881F991F5A95A9F780959095BC01CD01CD
:061070000895F894FFCF83
:0C1076004156524953505F320001010006
:00000001FF
